:020000040000FA
:1000000010280028002800288B0106288301831669
:10001000FF30860087000F308500831285000F288F
:1000200083018A01831640308F00831203179E01DB
:100030009F0103138316950116169616FF3085004F
:100040008601E0308700831291018F018E019001BB
:100050009012101210148B018C018D018501860104
:1000600087018030F100F000F201F301F401F501A5
:10007000F601F701F801F901FA01FB0101308F21C6
:1000800013308F2132308F2120308F218E1F462850
:100090008E1B48280C1C4E280C10910A6C21F0066F
:1000A000F000031D84287D21F106F100031D642862
:1000B0007008203A031D5E287108F5007008103A98
:1000C000031D64288721F600F01E6F28F20A7208CB
:1000D000313C03186D28F716F203F4017128F7126A
:1000E000F201701E7C28F30A7308313C03187A2849
:1000F0007716F303F4017E287712F301F40A031D47
:1001000083288030F90087288030F100F401F90855
:10011000031DFF28F71BBB28F71EA928F7189828EE
:100120001030B121F7147608FA00FF30FB00A62842
:100130007B08FF3A031D9F289030F900A528760818
:10014000FA007508FB001030B121F710F717910184
:10015000BA28F71CBA2876087A060319B028FB01DA
:10016000771CB4289030F90011081D3C0318BA28F8
:100170009030F900C428F71AC428F718C328771B51
:10018000C3281030F900F713771BF528771EE328F2
:100190007718D2281030B12177147608FA00FF3092
:1001A000FB00E0287B08FF3A031DD9289030F900B6
:1001B000DF287608FA007508FB001030B1217710AF
:1001C00077179101F428771CF42876087A0603192A
:1001D000EA28FB01F71CEE289030F90011081D3CBD
:1001E0000318F4289030F900FE28771AFE287718B3
:1001F000FD28F71BFD282030F90077130129F7139C
:10020000771378082C3C031C07291430B121780897
:1002100003190C29F8035D2979080F390F3A031DDA
:100220001529F7107710F9015D2979080F390E3A71
:10023000031D20290E30B121F7107710F9015D2937
:100240007908F039103A031D2E297708303903193F
:100250002C299030F9002D2913225D297908F039D5
:10026000203A031D3C297708303903193A29903088
:10027000F9003B29F0225D297908F039D03A031DB5
:100280004A2977083039031948299030F90049295B
:100290000D245D297908F039703A031D5129C621D2
:1002A0005D297908F039803A03195E297908F03917
:1002B000903A031D5D29CD215D2946288316051638
:1002C000851683121010F0308600870105088B1503
:1002D0000B10630000001028831605168516831284
:1002E00005083039FC008316051285128312770E3B
:1002F0003039303A85007C0808000708E039FC00F6
:100300000310FC0C05080F397C047F3A0800033009
:100310008A007108253E03188A0A82000628333AAB
:10032000FC008E018F010C1083160F3085008312A4
:100330000E080F02031D031C9F297C0EA0297C08B8
:1003400085000C1C98290C100800003A0319FF3096
:100350009E0008001D3003109E0D03189E061E0807
:100360000800FC00FC077C07FC07F03086008701D2
:100370007C08633C031C08005A30F80003308A00F4
:100380007C08A53E03188A0A82000628FB0A7B081F
:100390000319F9010F39B12108003030F705031DA9
:1003A00008000F30F9040800FB13831BFB177A0EBB
:1003B000203E84007B0C0F398404FB1A84178313BE
:1003C0007B1B831700087B1C000E0F398313FB1B5C
:1003D0008317FB130800FB08031DFA2905307A0276
:1003E000FC00FC07FC077C0E03178D0083168C13A2
:1003F000831203137B180D2A831603170C140000B5
:10040000000083120C088D0A0313031D0A2A031728
:100410008F0A0313FC007C0E102A03170C08031329
:100420000F39080008007908103A031D2B2A7A08B2
:100430000D3A031D1E2AD030F90008007A08093C45
:100440000318252A1E30F9000800FB011030B121E5
:10045000F714F90A08007908113A031D432A7A08AB
:10046000043C031C352AD4213C2A7A08093C031C8D
:100470003B2AEB213C2A122276060319412A7606F2
:10048000B121F90A08007908123A031D552AF7101C
:100490007B1CF7141230B121FB0A7B085F3C031868
:1004A000532AF90A542AF90308007908133A031D5C
:1004B000652A1030B121F7107A0E03390319622A28
:1004C000F907642A0F30F90408007908143A031D6B
:1004D0006E2A0130B1211730F90008007908153A69
:1004E000031D772A0A30B1211730F9000800790876
:1004F000163A031D7E2A0F30F90408007908173ACE
:10050000031D862AFA30F800F90A08007908183A1B
:10051000031D8E2AFA30F800F90A08007908193A02
:10052000031D972A1130B1210F30F90408001E3045
:10053000F9000800FB13831BFB177A0E203E840092
:100540007B0C0F398404FB1A841783137B1B8317DE
:1005500076080F397B18AF2A8000800EB02A8004FD
:100560008313FB1B83170800FB08031DC32A0530F8
:100570007A02FC00FC07FC077C0E03178D00831633
:100580008C138312031376080F397B18CC2A0317B8
:100590008C008C0E0313EE2A03170C0403130317AD
:1005A0008C0003130330FF00831603178C130C1504
:1005B00055308D00AA308D008C148C18DD2A0C115A
:1005C00083120C0883160C1483120C0603130319F0
:1005D000EB2AFF0BD42A03178D0A03130800080027
:1005E0007908203A031D012B7A08093C0318FB2ADD
:1005F0002E30F9000800FB0177141030B121F90A00
:1006000008007908213A031D222B7A08043C031CB8
:100610000B2B9A22122B7A08093C031C112BB422B3
:10062000122BEF227710FB0A7B085F3C03181D2B6F
:100630001030B1210F30F904212B1230B1217B1C75
:10064000771408002E30F90008000034003400341C
:1006500000340034003401340734003400340034F2
:1006600000340034003400340034003400340034EA
:1006700000340034003400340034003400340034DA
:1006800000340034003400340034003400340034CA
:1006900000340034003400340034003400340034BA
:1006A00000340034003400340034003400340034AA
:1006B0000034003400340034003400340C3400348E
:1006C000003400340034003400340034003400348A
:1006D000003400340034003400340034003400347A
:1006E0000034003400340034033400340034003467
:1006F000003400340034003400340034003400345A
:100700000234003400340D3400340034003400343A
:100710000034003400340434003400340034003435
:100720000034003405340034093400340F3400340C
:1007300000340034003400340A3400340E34003401
:1007400000340B34063400340834EF3086001030A7
:1007500087000800EF308600083087000800EF307F
:100760008600043087000800EF30860002308700E2
:100770000800DF308600103087000800DF30860078
:10078000083087000800DF3086000430870008004A
:10079000DF308600023087000800BF30860010304E
:1007A00087000800BF308600083087000800BF308F
:1007B0008600043087000800BF30860002308700C2
:1007C00008007F3086001030870008007F308600E8
:1007D0000830870008007F3086000430870008005A
:1007E0007F308600023087000800EF30860001303D
:1007F00087000800DF308600013087000800BF3026
:1008000086000130870008007F30860001308700B5
:100810000800F0308600870108007908D03A031DEF
:10082000152C0D30B121F90A08007908D13A031DC1
:10083000222C1130B121FF30FB000F08FA00A52156
:10084000F90A0800F71477100F087A06031D08004C
:10085000AA21DF3C03182D2CFB0A703940380F0702
:10086000FA007B080F39FC004224FB007C027B026B
:100870000318412C7B08023C031C412C0330B1219E
:100880007714080004308A007508493E03188A0A64
:1008900082000F34003401340F3402340F340F342B
:1008A00009340334003401340F3402340F340F346C
:1008B000093404340F340F340F340F340F340F3431
:1008C000093404340F340F340F340F340F340F3421
:1008D000093405340F340F340F340F340F340F3410
:1008E000093405340F340F340F340F340F340F3400
:1008F00009340F340F340F340F340F340F340F34E6
:1009000009340F340F340F340F340F340F340F34D5
:10091000093406340F340F340F340F340F340F34CE
:10092000093406340F340F340F340F340F340F34BE
:1009300009340F340F340F340F340F340F340F34A5
:1009400009340F340F340F340F340F340F340F3495
:1009500009340F340F340F340F340F340F340F3485
:1009600009340F340F340F340F340F340F340F3475
:100970000934083408340834083408340834083496
:100980000F34083408340834083408340834083480
:020990000F3422
:02400E00C400EC
:00000001FF
